:0600000002005B02329DCC
:03000B000230F6CA
:030013000230F6C2
:03001B0002002BB5
:0300230002315156
:10002B0032416C636F726E204D634272696465205E
:10003B00496E632E20536372697074204F53202DC9
:10004B002056657273696F6E20362E353220202054
:10005B00C2AF75D00075815675B81175A813787F2E
:10006B00E4F6D8FD758DFD758BFD758C88758A084A
:10007B007589217588047536887535087598C01291
:10008B0034DF7E007F409020007400F0A3DEFCDFA5
:10009B00FA75A0687800E2F52C75A0687802E2F595
:1000AB002DD2AFD28CD28E121FE69000001230D11F
:1000BB00FAA31230D1FBA31230D1FCA31230D1B46E
:1000CB00800040027480FD4C6018A31230D1F540C3
:1000DB00A31230D1A31230D1F54E900002121FBEE5
:1000EB006017903BCA122B257537287455F59978F4
:1000FB000000D8FDD20302019774AAF5997800008D
:10010B00D8FDC203903BDB122B25122AE37538284E
:10011B0090000F1230D1A2E79209122EED754520F7
:10012B00754400754B00754A30854E4FE54E605651
:10013B00900020A3A3D54FFB75A02E7800854E4FC2
:10014B001230D1F2A3081230D1F2A308B800020585
:10015B00A0D54FEC854E4F85458285448312137590
:10016B00A3A31230D1540F854B82854A83F0A3850C
:10017B00824B85834A854582854483A3A38582452B
:10018B00858344D54FD1122F90122EABD29C1201E6
:10019B00C21202193001F7C20112387D2003EFC2DF
:1001AB0091122DD1120BF8120F431210DA12139772
:1001BB00121398D29180D775D0089021007F5C7E66
:1001CB0002E0F5F0A3E0F8A3E0F9686034E5F05441
:1001DB007FB4000512021A8028B401051204B28004
:1001EB0020B402051202778018B40505120A468066
:1001FB0010B40905120B458008B40805120546809A
:10020B0000E5822406F5820FDEB775D0002222AC02
:10021B0083AD828F83898275D00075A0247800E02E
:10022B00FB75F000E425F0F5F00582E582650860CA
:10023B002DE0F208DBEF0582C5F003547FB5F01E0D
:10024B00858209902400E0FBA3D20A7538031213B0
:10025B00CE300B03122DD175D008898280067537ED
:10026B003C75D008E5828C838D82F02285820C85CB
:10027B00830DE50FC3945C23245BF50B850F8385FE
:10028B000982E030E70FB4F8005007850B827583C5
:10029B0025F0020498850B82758325E0B49000400D
:1002AB000EB4A0004053B4F0030203500204985460
:1002BB000FB540F8E50904B508030204AB850F83BD
:1002CB00F582E030E7030204981582E00509C39438
:1002DB003CB400005020902400F5F0E540F0A374EE
:1002EB0003F0A3E5F0F075D0007BFF902400D20A59
:1002FB001213CE75D008020498540FB540AEE50921
:10030B0004B508030204AB850F83F582E030E703E5
:10031B0002049860B41582E00509C3943CB4000054
:10032B005020902400F5F0E540F0A37402F0A3E513
:10033B00F0F075D0007BFF902400D20A1213CE751B
:10034B00D008020498E508C39509B40700500302CE
:10035B00047F850F83850982E0B47F4A0582E0B470
:10036B007F028003B5403F0582E0B402390582E08D
:10037B00B47F028008B410028003B430290582E0F8
:10038B00B40703020437B4010DE508C39509B4099A
:10039B0000506902047FB4060DE508C39509B40A41
:1003AB0000500602047F02046A0582E020E7F76032
:1003BB00F5B4210050F0F50B0582E020E7E805824B
:1003CB00E020E7E2F5F00582E020E7DA0354804510
:1003DB00F0F5F0858209902400E540F0A37428F035
:1003EB00A3E50B14F0A3E5F0F075D0007BFF902490
:1003FB0000D20A1213CE75D0080204980582E020B1
:10040B00E75DC3943075F00AA4F5F00582E020E7B0
:10041B004EC3943025F075F00AA4F5F00582E02068
:10042B00E73DC3943025F014F5F080090582E020F8
:10043B00E72DC3F5F00582E0B4F7248582099024FB
:10044B0000E540F0A37418F0A3E5F0F075D0007B45
:10045B00FF902400D20A1213CE75D00802049830F4
:10046B00E70302049375373C850B8275832574F77C
:10047B00F0020498850F83850982E020E70A058244
:10048B00E582B508F50204AB8582091509850C8256
:10049B00850D83E50904F0F5096508600302028701
:1004AB00850C82850D8322AC83AD8275D010E50857
:1004BB00B5090302053B850F83850982E00509B465
:1004CB00F5ECA8091509E508C398B405005003021B
:1004DB00053B1209EFB54045902400F0A3F5F0124F
:1004EB0009EFFBB40300503525F0F5F01209EF606E
:1004FB002CB440005027F925F0F5F0E92405FAE576
:10050B0008C39509FEB5120040261209EFF0A3258A
:10051B00F0F5F0D9F51209EFB5F002800875373C0C
:10052B0005090204B97538031209FF88090204B9D9
:10053B0075D008E5098C838D82F022AC83AD827572
:10054B00D010E508B5090302060F850F83850982D4
:10055B00E0B4F1028004050980E88509F005F0E5B7
:10056B0008B5F00875D0088C838D8222850F8385A2
:10057B00F082E0B4F10280DEB4F202800405F08078
:10058B00DEE508B5090302060F850F83850982E0B6
:10059B000509B4F10F74011209A575A02078C8E400
:1005AB00F202058CB4F2161209CC30E00AC2E0C29A
:1005BB00E11209A502061A75373C02058CF5F012FB
:1005CB0009CC20E00675373C02058CF8E5F0B4F059
:1005DB0009E8D2E11209A502058CE830E10BC2E172
:1005EB001209A5E5F024F0F5F075A02078C8E275A6
:1005FB00A033780028F8E5F0F2E80475A02078C85D
:10060B00F202058C75D008E5098C838D82F022757A
:10061B00A02078C8E2B40300500675373C0206B838
:10062B0075A033780028F818E2F5F0790018E22964
:10063B00F918B8FFF9E9B5F002800675373C0206E8
:10064B00B875A03378009020C41209501208E5B495
:10065B00000675373C0206B8B40121E49020B4F0D3
:10066B00A3F0A3F0A3F09020B8F0A3F0A3F0A3F0B5
:10067B009020BCF0A3F0A3F0A3F080129020B41252
:10068B0009509020B81209509020BC1209507900E3
:10069B00C0129020C8E0FA1AE4F5F0E2F30809055D
:1006AB00F0EAB510F6E5F0F0D0120206BB02060F29
:1006BB001208E5B402399020B4E0B4FF1AA3E0B4F9
:1006CB00FF15A3E0B4FF10A3E0B4FF0B1209CCD2CB
:1006DB00E31209A50206FA7582B4E0700FA3E0706D
:1006EB000BA3E07007A3E0B5400280030207C375BC
:1006FB00A03378009020C01209509020C0E0A3B422
:10070B000016E0A3B40011E0A3B4000CE0B40402A3
:10071B008009B4003B0207C00207C0E2B4003108F5
:10072B00E22403FEE2FE08902400E540F0A3E2F091
:10073B0008A3EEB510F890240075D000D20A7538D6
:10074B00031213CE75D0101209CC30E3090207C384
:10075B0075373C0207C075A02078C412090D12082A
:10076B00E5B4021475A02078B812090D75A0207895
:10077B00B412090D7405F0A3E4F0A37401F0A37592
:10078B00A02078C8E2F975A0337800E2F008A3E85E
:10079B00B511F875A024780075F000A982E2082540
:1007AB00F0F5F0E8B511F6E5F0F0A3E50FC3945CB6
:1007BB00FA0912088302082C9020BCE0700EA3E00B
:1007CB00700AA3E07006A3E07002805514F0B4FF2A
:1007DB00187582BEE014F0B4FF0F7582BDE014F003
:1007EB00B4FF067582BCE014F0E50FC3945CF5F022
:1007FB00902100E5822408F5827A01E0547FB40849
:10080B0016E5F0B51202800FAD82AE83AFF0120881
:10081B002F8D828E838FF0E5822408F5820ABA022F
:10082B00DA0206B890240075A02078C412090D7561
:10083B00A02078B412090D75A02078B812090D7597
:10084B00A02078BC12090D75A02078C8E2F975A01C
:10085B00337800E2F008A3E8B511F875A02478000E
:10086B0075F000A982E20825F0F5F0E8B511F6E580
:10087B00F0F0A3091208832290340074F1F0A375F1
:10088B00A0247800E208B4F007F0A3E4F0A3801CE6
:10089B00B4F10A74F0F0A37401F0A3800FB4F20A60
:1008AB0074F0F0A37402F0A38002F0A3E8B511D4A6
:1008BB0074F2F0A3A98290240075A0347800E2F0C2
:1008CB0008A3E582B511F775D000902400AB11AAEF
:1008DB0012D20A122BAE75D01022C082C083902088
:1008EB00C4E0B40016A3E0B40011A3E0B4000CA361
:1008FB00E0B401028007B4020280027400D083D0FE
:10090B008222E208601674FDF0A30808E218F0A337
:10091B00E218F0A3E218F0A3E2F0A322E2086011C0
:10092B0074FEF0A308E218F0A3E218F0A3E2F0A320
:10093B0022E208600C74FFF0A3E218F0A3E2F0A32C
:10094B0022E2F0A322C011E2F9B9FD17080808084A
:10095B00E218F0A3E218F0A3E218F0A3E2F0080803
:10096B00088033B9FE14E4F0A3080808E218F0A3DA
:10097B00E218F0A3E2F00808801CB9FF10E4F0A322
:10098B00F0A30808E218F0A3E2F0088009E4F0A352
:10099B00F0A3F0A3E2F008D01122C009C082C083FB
:1009AB00C0E0E50FC3945CF509902100E5822408B3
:1009BB00D509FB2407F582D0E0F0D083D082D00993
:1009CB0022C009C082C083E50FC3945CF509902156
:1009DB0000E5822408D509FB2407F582E0D083D0FB
:1009EB0082D00922C083C082850F838882E008D021
:1009FB0082D0832275D0007BFF902400D20A121381
:100A0B00CEE513B40002802FB40214E50FC3945C3F
:100A1B00FA850F83850982E516FBD20A122BAEE508
:100A2B000FC3945CFA74AA3012027455902400F030
:100A3B007B01D20A122BAE75D01022AC83AD82751E
:100A4B00D010A809E508C398B40C005003020B3A68
:100A5B00850F83E5092402F582E0B43A028066B47F
:100A6B002D60A809E508C398B417005003020B3A90
:100A7B00E5092416F582E0B40D48902400A8097905
:100A8B0019120B9B120BCB08791A120B9B120BCB67
:100A9B0008791B120B9B120BCBE82406F8791C125E
:100AAB000B9B120BCB08791D120B9B120BCB0879EE
:100ABB001E120B9B120BCB791FE4120BCBE8F50923
:100ACB008080020B35E509240BF582E0B40D5BA8A1
:100ADB0009E8F9120B9BB41800504C1209EFB43A09
:100AEB0046120B9BB43C00503E1209EFB43A38123D
:100AFB000B9BB43C005030753803902400E9F87917
:100B0B001C120B9B120BCB08791D120B9B120BCBE0
:100B1B0008791E120B9B120BCB791FE4120BCBE542
:100B2B0009240CF509414D75373C0509020A4D7531
:100B3B00D008E5098C838D82F022AC83AD8275D011
:100B4B0010A809E508C398B405004039850F8385C3
:100B5B000982E0B4432AA809E5092403F8E8120B3B
:100B6B009B601AB46300501514758330F582E0D284
:100B7B00E2F0753803E5092405F50980C475373CA7
:100B8B000509020B4C75D008E5098C838D82F02288
:100B9B00C083C082850F838882E0080582C39430AE
:100BAB00B40600501475F00AA4F5F0E008C39430B5
:100BBB00B40A00500425F0800274FFD082D0832247
:100BCB00C0F0F5F0E540F0A37428F0A3E9F0A3E53D
:100BDB00F0F0A324282903547FF075D0007BFF90FD
:100BEB002400D20A1213CE75D010D0F022906800D8
:100BFB00E09039BC93F8C52C6830E00CC0E0A260E3
:100C0B0075F000120CF9D0E030E10CC0E0A2617578
:100C1B00F001120CF9D0E030E20CC0E0A26275F0EA
:100C2B0002120CF9D0E030E30CC0E0A26375F003C4
:100C3B00120CF9D0E030E40CC0E0A26475F00412A1
:100C4B000CF9D0E030E50CC0E0A26575F005120C94
:100C5B00F9D0E030E60CC0E0A26675F006120CF994
:100C6B00D0E030E708A26775F007120CF990680224
:100C7B00E09039BC93F8C52D6830E00CC0E0A26859
:100C8B0075F008120CF9D0E030E10CC0E0A26975E8
:100C9B00F009120CF9D0E030E20CC0E0A26A75F05A
:100CAB000A120CF9D0E030E30CC0E0A26B75F00B2C
:100CBB00120CF9D0E030E40CC0E0A26C75F00C1211
:100CCB000CF9D0E030E50CC0E0A26D75F00D120C04
:100CDB00F9D0E030E60CC0E0A26E75F00E120CF904
:100CEB00D0E030E708A26F75F00F120CF9229205D5
:100CFB0090257DE07003020E5BF54F754D00754C32
:100D0B0026854D82854C83E0F9A3E0FAA3E0A3A3EB
:100D1B0085824D85834C89828A83F545C0F075F0B9
:100D2B0002A4F54B85F04AD0F0A3A31230D1FBA35C
:100D3B001230D1FCA31230D1FDA31230D1FEA3127D
:100D4B0030D1FFEF547FB5F05EEB20E40520055763
:100D5B008003300552EE600CB407005007120E5F93
:100D6B0040028043903000E5452582F582E030E279
:100D7B003030E02FE54B2400F582E54A3431F58322
:100D8B00121388E582C39CE5839D5003020E58E540
:100D9B0045121D12758330854582E0D2E2F0020EBA
:100DAB0058D2E2F0020E58A31230D1FEA31230D16A
:100DBB00FFEF547FB5F02BEB20E5052005248003D6
:100DCB0030051FEE600CB407005007120E5F400297
:100DDB008010903000E5452582F582E0C2E2F002FA
:100DEB000E58A31230D1FEA31230D1FFEF547FB5B2
:100DFB00F02BEB20E605200524800330051FEE6069
:100E0B000CB407005007120E5F40028010903000A8
:100E1B00E5452582F582E0D2E3F0020E58A31230AD
:100E2B00D1FEA31230D1FFEF547FB5F020EB20E7BA
:100E3B00052005198003300514EE600CB407005033
:100E4B0007120E5F40028005E545121D12D54F01BA
:100E5B0022020D0CC082C083C0F0E5822407F5820C
:100E6B00E5833400F5831230D1F8A31230D1541F2F
:100E7B00240BF975A025E3F9EE30E708E8541F249D
:100E8B000BF8E2F8EE540F2323900E9873020ED852
:100E9B0000020EDC00020EEA00020EF800020F0840
:100EAB0000020F1A00020F2A00020EDC00020EEAEB
:100EBB0000020EF800020F0800020F1A00020F2AA0
:100ECB0000020ED800020ED800020ED800C3020F8B
:100EDB003CE988F0B5F004D3020F3CC3020F3CE9A8
:100EEB0088F0B5F004C3020F3CD3020F3CE988F045
:100EFB00B5F0004004C3020F3CD3020F3CE988F06D
:100F0B00B5F00280064004C3020F3CD3020F3CE84D
:100F1B0089F0B5F00040E2C3020F3CD3020F3CE86E
:100F2B0089F0B5F00280064004C3020F3CD3020FD8
:100F3B003CD0F0D083D08222200F03021072902578
:100F4B007EE07003021072F54F754D00754C2A85CB
:100F5B004D82854C83E0F9A3E0FAA3E0A3A385823D
:100F6B004D85834C89828A83F545C0F075F002A4C8
:100F7B00F54B85F04AD0F0A3A31230D1FBA312306E
:100F8B00D1FCA31230D1FDA31230D1FEA31230D16C
:100F9B00FFEE541FB40700404A1210754002804305
:100FAB00903000E5452582F582E030E23030E02FCD
:100FBB00E54B2400F582E54A3431F583121388E5BD
:100FCB0082C39CE5839D500302105EE545121D1202
:100FDB00758330854582E0D2E2F002105ED2E2F0FA
:100FEB0002105EA31230D1FEA31230D1FFEE541FBC
:100FFB00B40700401712107540028010903000E5C6
:10100B00452582F582E0C2E2F002105EA31230D1D8
:10101B00FEA31230D1FFEE541FB40700401712107D
:10102B007540028010903000E5452582F582E0D2B4
:10103B00E3F002105EA31230D1FEA31230D1FFEE0B
:10104B00541FB40700400C12107540028005E54593
:10105B00121D12D54F03021067020F5A7E209025E6
:10106B002B7400F0A3DEFCC20F22C082C083C0F041
:10107B00E5822407F582E5833400F5831230D1F83D
:10108B00A31230D1541FF990252B2582F582E0C293
:10109B00046002D204EE30E719E8541FF890252BB8
:1010AB002582F582E06002D20475A025740B28F826
:1010BB00E2F830041275A025740B29F9E3F9EE540C
:1010CB000F2323900E9873C3D0F0D083D082228548
:1010DB004E4FE54E7003021333754B00754A307556
:1010EB004D00754C2E900020E54E12133A85824729
:1010FB0085834675430075423175452075440085DF
:10110B004B82854A83E020E2030212C990001C1235
:10111B0030D15401700890001B1230D160328545DC
:10112B008285448312137574152582F582740035FC
:10113B0083F5831230D130E017C082C08320E104E5
:10114B00740080027401903504F0D083D08280113A
:10115B00C082C0837400903504F0D083D082021219
:10116B0042A31230D1F8A31230D1F9A31230D1FA25
:10117B00903502E0FB903501E0FC903500E0FDC3BB
:10118B00EB98F582EC99F5838542A0A843E582F2B2
:10119B0008E583F2ED9A30E7030212307071903557
:1011AB0005854FF0C3E58225F0F582E5833400F524
:1011BB0083E020E211E2701718E275F005B5F0023A
:1011CB00800440028009903503E0700302125890AE
:1011DB003504E0700302128985478285468312131A
:1011EB0075858249858348121375E5824583601F97
:1011FB0012134D600A854982854883A3A380E2853B
:10120B004D82854C83E549F0A3E548F00212BC9072
:10121B003504E06069854D82854C83E549F0A3E593
:10122B0048F00212BC85478285468312137585826E
:10123B00498583480212BC854382854283121388F9
:10124B00A38542A0A843E582F208E583F2854D828F
:10125B00854C83121388858249858348121375E563
:10126B00824583601912134D6047A3A3C20A121360
:10127B00CE20063D854982854883A3A380D890352F
:10128B0004E0702D8547828546831213758582494C
:10129B008583488542A0A8437400F208F2854B82EF
:1012AB00854A83E030E10510E3028002C2E2C2E42A
:1012BB00F0854D82854C83E549F0A3E548F0854BDD
:1012CB0082854A83E0F9903505854FF0C3E5822589
:1012DB00F0F582E5833400F583E9F0D54F028048C1
:1012EB00854B82854A83A385824B85834A854D82B4
:1012FB00854C83A3A385824D85834C854782854688
:10130B0083A3A3858247858346854382854283A336
:10131B00A3858243858342854582854483A3A38528
:10132B00824585834402110A9035037400F022C074
:10133B00F075F002A42582F582E5F03583F583D0B4
:10134B00F022AD82AE83121375AB82AC83854382E0
:10135B00854283121388E582C39BE5839C4004740A
:10136B00FF800274008D828E8322C0F01230D1F583
:10137B00F0A31230D1F58385F082D0F022C0F0E0DB
:10138B00F5F0A3E0F58385F082D0F0222230133202
:10139B00E550B4022D14F550780075A02574FFF2BA
:1013AB0008E540F2087400F208E52CF208E52DF28E
:1013BB0008E52EF208E52FF29025007A007B2B1220
:1013CB002BAE22C206AD82AE837A001230DDFFA3B4
:1013DB001230DDC212B467004003D21222903ABC25
:1013EB0075F002A42582F582E5F03583F583E4934D
:1013FB00F5F0A3E49385F083F582E4731215B6023E
:10140B0015B11215CC0215B11215E20215B1121558
:10141B00E30215B11215E40215B11215FA0215B15A
:10142B001216090215B11216480215B112166002F6
:10143B0015B11216780215B11216A10215B11217B9
:10144B00F80215B1122E730215B11218560215B10E
:10145B0012189D0215B11219C00215B1121AE3022E
:10146B0015B1121B1A0215B1121B660215B1121B14
:10147B00B20215B1121C0C0215B1121AF80215B1F9
:10148B00121C660215B1121CCC0215B1121CE5021E
:10149B0015B1121CFE0215B1121E330215B1121F2B
:1014AB00440215B112216C0215B11235120215B19D
:1014BB00122AE30215B1122B030215B11221C2023B
:1014CB0015B11221C30215B112220B0215B1122252
:1014DB002F0215B112225B0215B11222880215B12F
:1014EB001222B90215B11222E80215B112231B0206
:1014FB0015B112234C0215B11223860215B112231A
:10150B00C10215B11224000215B112243D0215B10E
:10151B0012247E0215B11224BD0215B11224E4026D
:10152B0015B112250D0215B11225390215B112256F
:10153B006A0215B112259D0215B11225D40215B1FF
:10154B001226090215B11226420215B11226790292
:10155B0015B11226B80215B11226F90215B11227D0
:10156B003E0215B11227810215B11227C80215B11F
:10157B0012280D0215B112283C0215B11221C4021A
:10158B0015B11221C50215B112286D0215B1122821
:10159B00F60215B112292C0215B1122ACD0215B182
:1015AB0012296B0215B18D828E83228D828E83A3BD
:1015BB00A31230DD543F2474F58275832074FFF041
:1015CB00228D828E83A3A31230DD543F2474F582C7
:1015DB007583207400F02222228D828E83A3A312A6
:1015EB0030DD543F2474F582758320E0F4F0228DB6
:1015FB00828E83A3A31230DDFBA312204422902200
:10160B0000E0F8A3E0F5F075A05E902100E0547FB8
:10161B00B4010579010216257900903B8CE99360A2
:10162B000BF20908E8B5F0F5D2068010902200E81D
:10163B00C2ACF0200804D208D299D2AC228D828E93
:10164B0083A3A31230DDFAA31230DDFBA3122BAE62
:10165B006002D206228D828E83A3A31230DDFAA301
:10166B001230DDFBA3122C296002D206228D828E52
:10167B0083A3A31230DDFA7B01A31230DD90250B7F
:10168B002582F582A20AC0D0D20A122BAED0D092FC
:10169B000A6002D206228D828E83A3A31230DDFA5A
:1016AB00A31230DDC0E0A31230DDFF5407232390DB
:1016BB0016BE730216DD0002170F0002173A000266
:1016CB00175F000216DD000216DD000216DD0002B8
:1016DB0016DDD0E090250B2582F582E078007900AD
:1016EB007C00600F75F00A84A8F0600775F00A841F
:1016FB00A9F0FCE82430F8E92430F9EC2430FC7B29
:10170B000302177DD0E090250B2582F582E0540F64
:10171B002430B43A0040022407F9E054F0C42430DA
:10172B00B43A0040022407FC78207B0202177DD0DC
:10173B00E090250B2582F582E054072430F8E05425
:10174B00380303032430F9E054C023232430FC7BFB
:10175B000302177DD0E090250B2582F5827B01A239
:10176B000AC0D0D20A122BAED0D0920A607ED2061B
:10177B00807AEF543803901785730217A400021771
:10178B00D8000217C9000217B2000217A4000217F3
:10179B00A4000217A4000217A4BB0102802FBC30C7
:1017AB002CE9FCE8F9DBF2BC3023E9FCE8F9782002
:1017BB00BB031ABC3017E9FCE8F97820800FBC306A
:1017CB000C7C20BB0307B9300479208000902044A7
:1017DB00ECF0A3E9F0A3E8F0902044A20AC0D0D229
:1017EB000A122BAED0D0920A6002D206228D828EC4
:1017FB0083A3A31230DDFAA31230DDF8A31230DD80
:10180B00F9A31230DD90250B2582F582E0FB9020A9
:10181B00447406F0A3E5404480F0FCA3E8F02CFCF4
:10182B00A37428F02CFCA3E9F02CFCA3EBF02CA365
:10183B0003547FF09020447B07A20AC0D0D20A1237
:10184B002BAED0D0920A6002D206228D828E837587
:10185B00D010A3A31230DDFBA3AD82AE8390210089
:10186B00E5822408F5827A01E0547FB40819A88236
:10187B00A9838D828E8375D000AA12AB13122BAE67
:10188B0075D01088828983E5822408F5820ABA0212
:10189B00D722854B82854A83E0F98D828E83A3A361
:1018AB001230DDFA232323FC75A021F8E920E44252
:1018BB00E2C2E7F2E408F208F2A31230DDFBA31256
:1018CB002BAE75A021ECF8E2D2E7F2080808080865
:1018DB001230DDF2A3081230DDF2200606A3081247
:1018EB0030DDF2854B82854A83E0D2E4F0D20602EA
:1018FB0019BF08A31230DD24052582F582E4358358
:10190B00F5831230DDF5F0E2C395F0501E080808A0
:10191B0008E2F5F008E245F0602D18E2C39401F2FD
:10192B00500408E214F2D2060219BFABF0A3EA246A
:10193B005CF5A078001230DDF5F0E2B5F009A308F4
:10194B00DBF3753803804A75A021EC2407F8E260BD
:10195B000F14F28D828E83A3A3ECF8D2060218BB70
:10196B0075373C30092B9000141230D1F8A312308C
:10197B00D1F5838882E5822AF582E43583F58312DB
:10198B0030D1F8C3954E50097583308882E0D2E28E
:10199B00F075A021ECF8E2547FB403028003B40786
:1019AB0004C2E78002D2E7F2854B82854A83E0C20C
:1019BB00E4F0C20622854B82854A83E0F98D828E44
:1019CB0083A3A31230DDFA232323FC75A021F8E9AE
:1019DB0020E442E2C2E7F2E408F208F2A31230DD9F
:1019EB00FBA3122C2975A021ECF8E2D2E7F2080830
:1019FB000808081230DDF2A3081230DDF2200606CB
:101A0B00A3081230DDF2854B82854A83E0D2E4F0E5
:101A1B00D206021AE208A31230DD24052582F582D4
:101A2B00E43583F5831230DDF5F0E2C395F0501EFB
:101A3B0008080808E2F5F008E245F0602D18E2C34B
:101A4B009401F2500408E214F2D206021AE2ABF04F
:101A5B00A3EA245CF5A078001230DDF5F0E2B5F0D6
:101A6B0009A308DBF3753803804A75A021EC240722
:101A7B00F8E2600F14F28D828E83A3A3ECF8D206EA
:101A8B000219DE75373C30092B9000141230D1F857
:101A9B00A31230D1F5838882E5822AF582E435835F
:101AAB00F5831230D1F8C3954E5009758330888277
:101ABB00E0D2E2F075A021ECF8E2547FB40302808F
:101ACB0003B40704C2E78002D2E7F2854B82854A52
:101ADB0083E0C2E4F0C206228D828E83A3A3123070
:101AEB00DD547F232549F54950020548228D828E0E
:101AFB0083A3A31230DDFAA31230DDF9EAC333FA64
:101B0B00E933F9EAC32549F549E93548F548228D0A
:101B1B00828E83A3A31230DD20E71810E60A121F72
:101B2B00A4B900047824801E2474F875A020E270F8
:101B3B001A8027547F121FA4B90004782C8007B990
:101B4B000104782D8000567002800FA31230DD54F3
:101B5B007F232549F54950020548228D828E83A3A8
:101B6B00A31230DD20E71810E60A121FA4B90004F7
:101B7B007824801E2474F875A020E2601A80275404
:101B8B007F121FA4B90004782C8007B90104782DAB
:101B9B008000566002800FA31230DD547F2325494D
:101BAB00F54950020548228D828E83A3A31230DDA6
:101BBB0020E71810E60A121FA4B900047824801E2F
:101BCB002474F875A020E2701A8035547F121FA47C
:101BDB00B90004782C8007B90104782D8000567069
:101BEB0002801DA31230DDFAA31230DDF9EAC333F4
:101BFB00FAE933F9EAC32549F549E9FA3548F548D5
:101C0B00228D828E83A3A31230DD20E71810E60A03
:101C1B00121FA4B900047824801E2474F875A02028
:101C2B00E2601A8035547F121FA4B90004782C800F
:101C3B0007B90104782D8000566002801DA3123075
:101C4B00DDFAA31230DDF9EAC333FAE933F9EAC35B
:101C5B002549F549E9FA3548F548228D828E83A34B
:101C6B00A31230DDF8C3954E50567583308882E051
:101C7B0030E24A30E04AC004C005900020E812135D
:101C8B003A121375A3A3A31230D1FCA31230D1FDCA
:101C9B00E8C0F075F002A42400F582E5F03431F5CC
:101CAB0083D0F0121388E582C39CE5839DD005D0C9
:101CBB0004400DE8121D127583308882E0D2E2F0E9
:101CCB00228D828E83A3A31230DDF8C3954E50096B
:101CDB007583308882E0C2E2F0228D828E83A3A3CB
:101CEB001230DDF8C3954E50097583308882E0D2EF
:101CFB00E3F0228D828E83A3A31230DDF8C3954EC1
:101D0B005004E8121D1222C000C003C004C0F0F83A
:101D1B00900020E54E12133AE812133A121375ABEA
:101D2B0082AC8375832EE875F002A4F582E5F0355D
:101D3B0083F583EBF0A3ECF0758331E875F002A427
:101D4B00F582E5F03583F583E4F0A3F075833088F5
:101D5B0082E0C2E2C2E4F0C2E3D0F0D004D003D000
:101D6B000022902200E0F875A05E902100E0547FE5
:101D7B00B400047402F2089000021230D1A3F208EE
:101D8B001230D1F208902200E8C2ACF0200804D245
:101D9B0008D299D2AC22C004C005C00675A0257824
:101DAB004B791075040075050075060CD5041DD50F
:101DBB00051AD506177455C29BC299F5997504007F
:101DCB00750504D504FDD505FA02005B3098DDE5F9
:101DDB0099F2C298EA70011B1AEB7003EA601108C2
:101DEB00D9C1784B7910E21230C1A308D9F880AC75
:101DFB007A007B20DAFEDBFC784B7910E21230C1E3
:101E0B00A308D9F8902100E0547FB4011474AAC23E
:101E1B009BC299F599750400750508D504FDD50588
:101E2B00FAD006D005D00422C2AF8D828E83A3A335
:101E3B001230DDFAA31230DDFBE599C29874AAC209
:101E4B009BC299F599900000121DA102005B8D8237
:101E5B008E83A3A31230DDFAA31230DDFB900002B8
:101E6B001230D1F8A31230D1C854F0241CC8500141
:101E7B0004F5838882745A1230C1A374A51230C141
:101E8B00A3EA1230C1A3EB1230C1A3C000C001758D
:101E9B000000750100D500FDD501FAD001D000C2BC
:101EAB00AFE599C29874AAC29BC299F599121DA16C
:101EBB0074AAC29BC299F599750400750504D504E3
:101ECB00FDD505FA02005B2014FDC29BD214F599D7
:101EDB00229000021230D1F8A31230D1C854F02452
:101EEB001CC8500104F58388821230D1B45A18A350
:101EFB001230D1B4A511A31230D1FAA31230D1FBF9
:101F0B00A3BA000CBB0009E4121ED2121ED2801A17
:101F1B00EA121ED2EB121ED21230D1A3121ED21A0B
:101F2B00BAFF011BBA00F1BB00EE75040075050486
:101F3B00D504FDD505FA02005B9000021230D1FAF0
:101F4B00A31230D1FB700CEA7009E4121ED2121EE0
:101F5B00D280278A828B83A3A3AA82AB83EA121E29
:101F6B00D2EB121ED29000001230D1A3121ED21A45
:101F7B00BAFF011BBA00F1BB00EE75040075050436
:101F8B00D504FDD505FA02005B8D828E83A3A312C7
:101F9B0030DDC2136002D21322F95407C9030303C5
:101FAB005403C0E07401B90002800323D9FDF9D0BA
:101FBB00E0C922780079001230D128500109F8A32A
:101FCB00DC05BD00F28006BCFFED1D80EAE86A70FF
:101FDB0007E96B7003E4800274FF2290000075A088
:101FEB00787802E230E70BA3E583B405F6C2110261
:101FFB002043D2117A30122B497A30122B497A387E
:10200B00122B497A80122B497A06122B497A0C1221
:10201B002B497A01122B497A40122B497A5A122BEF
:10202B00687A40122B49122B8AB45AC1903BB912D1
:10203B002B25903BA0122B3722EB60627A80122B60
:10204B00491230DDB404005029A3DB028050B400E8
:10205B00047A808010B401047AC08009B402047A37
:10206B009480027AD41230DDA3543F2AFA122B4902
:10207B00802AB40C08A37A01122B49801FB40D03DC
:10208B00A38014B40A03A3800EB40E2EDB11800EB2
:10209B00FA122B68A380057AC0122B49DBA322A36B
:1020AB001230DD14A3C082C08390250B2582F582EC
:1020BB00E0D083D08212212880E2B40FD3DB0280E0
:1020CB00DDA31230DD14A3C082C08390250B2582C3
:1020DB00F582E0D083D0821220E780C07C017A2089
:1020EB00C39464400C1C7A31C394644004C394645D
:1020FB000A2464C0E0122B68D0E07A31C3940A4002
:10210B00030A80F81A240AC0E0BA3005EC60027AA0
:10211B0020122B68D0E02430FA122B68227C017A33
:10212B0020C39464400C1C7A31C394644004C39460
:10213B00640A2464BA20028007C0E0122B68D0E046
:10214B007A31C3940A40030A80F81A240AC0E0BA11
:10215B003003EC7003122B68D0E02430FA122B689A
:10216B00228D828E83A3A31230DD5403FB70059066
:10217B003BEC8013B40105903BFC800BB402059043
:10218B003C0C8003903C1C7A01122B497C10E4938D
:10219B00FA122B68A3DCF77C107AC0122B49EBC424
:1021AB002474F582758320E060047A3180027A30E2
:1021BB00122B68A3DCF1222222228D828E83A3A311
:1021CB001230DDFAA31230DDFBEA701875A025740E
:1021DB000B2BF8E52CF275A025742B2BF874FFF262
:1021EB00D20F801BB4011875A025740B2BF8E52DAD
:1021FB00F275A025742B2BF874FFF2D20F800022FE
:10220B008D828E83A3A31230DD541FF9240BF8A308
:10221B001230DD75A025F275A025742B29F874FFFB
:10222B00F2D20F228D828E83A3A31230DD541FF9BD
:10223B00240BF875A025E2F5F0A31230DDB5F00FF5
:10224B00A31230DD547F232549F54950020548225E
:10225B008D828E83A3A31230DD541F240BF875A03F
:10226B0025E2F5F0A31230DDB5F002800FA312309A
:10227B00DD547F232549F54950020548228D828E76
:10228B0083A3A31230DD541F240BF875A025E2F5B0
:10229B00F0A31230DDC5F0B5F0004002800FA312A1
:1022AB0030DD547F232549F54950020548228D82A4
:1022BB008E83A3A31230DD541F240BF875A025E2E7
:1022CB00F5F0A31230DDB5F0004002800FA3123001
:1022DB00DD547F232549F54950020548228D828E16
:1022EB0083A3A31230DD541F240BF875A025E2F550
:1022FB00F0A31230DDC5F0B5F00280044002800F70
:10230B00A31230DD547F232549F54950020548229D
:10231B008D828E83A3A31230DD541F240BF875A07E
:10232B0025E2F5F0A31230DDB5F002800440028007
:10233B000FA31230DD547F232549F5495002054880
:10234B00228D828E83A3A31230DD541FF9240BF848
:10235B0075A025E2F5F0A31230DDB5F01DA3123008
:10236B00DDFAA31230DDF9EAC333FAE933F9EAC334
:10237B002549F549E9FA3548F548228D828E83A324
:10238B00A31230DD541F240BF875A025E2F5F0A342
:10239B001230DDB5F002801DA31230DDFAA312302E
:1023AB00DDF9EAC333FAE933F9EAC32549F549E91B
:1023BB00FA3548F548228D828E83A3A31230DD5463
:1023CB001F240BF875A025E2F5F0A31230DDC5F044
:1023DB00B5F0004002801DA31230DDFAA31230DDF0
:1023EB00F9EAC333FAE933F9EAC32549F549E9FABE
:1023FB003548F548228D828E83A3A31230DD541FFE
:10240B00240BF875A025E2F5F0A31230DDB5F00032
:10241B004002801DA31230DDFAA31230DDF9EAC3AE
:10242B0033FAE933F9EAC32549F549E9FA3548F5B1
:10243B0048228D828E83A3A31230DD541F240BF808
:10244B0075A025E2F5F0A31230DDC5F0B5F00280E2
:10245B00044002801DA31230DDFAA31230DDF9EA2D
:10246B00C333FAE933F9EAC32549F549E9FA3548A3
:10247B00F548228D828E83A3A31230DD541F240BCB
:10248B00F875A025E2F5F0A31230DDB5F00280045B
:10249B004002801DA31230DDFAA31230DDF9EAC32E
:1024AB0033FAE933F9EAC32549F549E9FA3548F531
:1024BB0048228D828E83A3A31230DD541FF9240B87
:1024CB00F875A025E2FAA31230DD2AF275A0257467
:1024DB002B29F974FFF3D20F228D828E83A3A312C3
:1024EB0030DD541FF9240BF875A025E2FAA3123046
:1024FB00DDCAC39AF275A025742B29F974FFF3D2A8
:10250B000F228D828E83A3A31230DD541FF5F0248E
:10251B000BF8A31230DD541F240BF975A025E3F241
:10252B0075A025742B25F0F874FFF2D20F228D8243
:10253B008E83A3A31230DD541F240BF875A025E264
:10254B00F5F0A31230DD541F240BF9E3B5F00FA304
:10255B001230DD547F232549F54950020548228D61
:10256B00828E83A3A31230DD541F240BF875A02594
:10257B00E2F5F0A31230DD541F240BF9E3B5F002A2
:10258B0080DCA31230DD547F232549F54950020529
:10259B0048228D828E83A3A31230DD541F240BF8A7
:1025AB0075A025E2F5F0A31230DD541F240BF9E3DF
:1025BB00C5F0B5F0004002800FA31230DD547F232D
:1025CB002549F54950020548228D828E83A3A3121B
:1025DB0030DD541F240BF875A025E2F5F0A3123063
:1025EB00DD541F240BF9E3B5F0004002800FA3125A
:1025FB0030DD547F232549F54950020548228D8251
:10260B008E83A3A31230DD541F240BF875A025E293
:10261B00F5F0A31230DD541F240BF9E3C5F0B5F030
:10262B000280044002800FA31230DD547F23254922
:10263B00F54950020548228D828E83A3A31230DD0B
:10264B00541F240BF875A025E2F5F0A31230DD54CE
:10265B001F240BF9E3B5F00280044002800FA31294
:10266B0030DD547F232549F54950020548228D82E0
:10267B008E83A3A31230DD541F240BF875A025E223
:10268B00F5F0A31230DD541F240BF9E3B5F01DA3B5
:10269B001230DDFAA31230DDF9EAC333FAE933F96C
:1026AB00EAC32549F549E9FA3548F548228D828E6A
:1026BB0083A3A31230DD541F240BF875A025E2F57C
:1026CB00F0A31230DD541F240BF9E3B5F00280DCCC
:1026DB00A31230DDFAA31230DDF9EAC333FAE93382
:1026EB00F9EAC32549F549E9FA3548F548228D82BF
:1026FB008E83A3A31230DD541F240BF875A025E2A3
:10270B00F5F0A31230DD541F240BF9E3C5F0B5F03F
:10271B00004002801DA31230DDFAA31230DDF9EA6E
:10272B00C333FAE933F9EAC32549F549E9FA3548E0
:10273B00F548228D828E83A3A31230DD541F240B08
:10274B00F875A025E2F5F0A31230DD541F240BF928
:10275B00E3B5F0004002801DA31230DDFAA3123066
:10276B00DDF9EAC333FAE933F9EAC32549F549E957
:10277B00FA3548F548228D828E83A3A31230DD549F
:10278B001F240BF875A025E2F5F0A31230DD541FC2
:10279B00240BF9E3C5F0B5F00280044002801DA3C1
:1027AB001230DDFAA31230DDF9EAC333FAE933F95B
:1027BB00EAC32549F549E9FA3548F548228D828E59
:1027CB0083A3A31230DD541F240BF875A025E2F56B
:1027DB00F0A31230DD541F240BF9E3B5F002800493
:1027EB004002801DA31230DDFAA31230DDF9EAC3DB
:1027FB0033FAE933F9EAC32549F549E9FA3548F5DE
:10280B0048228D828E83A3A31230DD541FF5F02452
:10281B000BF875A025E2FAA31230DD541F240BF937
:10282B00E32AF275A025742B25F0F874FFF2D20F72
:10283B00228D828E83A3A31230DD541FF5F0240B5F
:10284B00F875A025E2FAA31230DD541F240BF9E32F
:10285B00CAC39AF275A025742B25F0F874FFF2D237
:10286B000F228D828E83A3A31230DD541FF9903C6F
:10287B002C7A01122B497C10E493FA122B68A3DCFF
:10288B00F77AC0122B499024007420F0A3F0A3F028
:10289B00A3F0A3E904122A65EBB430027420F0A371
:1028AB00EAF0A37420F0A3743DF0A37420F0A37599
:1028BB00A025E9240BF9E3122A65ECD204B4300409
:1028CB00C2047420F0A3EBB430052004027420F092
:1028DB00A3EAF0A37420F0A3F0A3F0A3F07C109074
:1028EB002400E0FA122B68A3DCF8228D828E83A3DE
:1028FB00A31230DD541FF9FB75A025240BF9E3FA65
:10290B0090001A1230D1C39401B408005012C423A2
:10291B00441FF583EB44E0F582EA1230C1122AD84A
:10292B00228D828E83A3A31230DD541FF990001ADF
:10293B001230D1C39401B408005024C423441FF5B2
:10294B0083E944E0F5821230D1FA75A025740B2986
:10295B00F8EAF275A025742B29F874FFF2D20F2236
:10296B00C0F08D828E83A3A31230DD75F03CA4FEE4
:10297B00AFF0A31230DDC32EFEEF3400FFA31230F5
:10298B00DD75F03CFB7C007D00C3EB2EFBEC3FFCCC
:10299B00ED3400FD15F0E5F070EFA31230DDF879A2
:1029AB00007A009000091230D1B4000575F0188040
:1029BB0013B4030575F019800BB4010575F01E8077
:1029CB000375F01EC3E82BF8E93CF9EA3DFA15F064
:1029DB00E5F070F09000091230D1B4013AEF700BB2
:1029EB00EE6034B40A030229F64018C3EE940AFED3
:1029FB00EF9400FFC3E89412F8E99400F9EA94000D
:102A0B00FA80DAC3EE9401FEC3E89402F8E994006D
:102A1B00F9EA9400FA80C6903500E0FD903501E0AC
:102A2B00FC903502E0FBC3E89BFFE99C7014EA9D28
:102A3B00701090001B1230D1F5F0EFB5F00280084A
:102A4B0040069035037401F0903500EAF0903501A3
:102A5B00E9F0903502E8F0D0F0227A007B007C00A0
:102A6B00601675F00A84AAF0600E75F00A84ABF05C
:102A7B00600675F00A84ACF0EA2430FAEB2430FBE4
:102A8B00EC2430FC229000001230D1FB902000127D
:102A9B0030D1FDEBF41230C1122AD81230D1F4B57B
:102AAB00030E9000001230D1B503057A20022ABD27
:102ABB007A08902000ED1230C1122AD890257FEAB7
:102ACB00F022122A9090257FE0FAF599227C00756E
:102ADB00F032DCFED5F0FB227A80122B497B28905A
:102AEB002580122B8AF0A3DBF97AC0122B497B28A5
:102AFB00122B8AF0A3DBF9227A80122B497B2890C8
:102B0B002580E0FA122B68A3DBF87AC0122B497BE5
:102B1B0028E0FA122B68A3DBF8227A80122B497477
:102B2B0000936007FA122B68A380F4227AC0122B51
:102B3B00497400936007FA122B68A380F422C0F04B
:102B4B0030111775F00075A0787802E230E70700B6
:102B5B00D5F0F3022B657800EAF2D0F022C0F0300A
:102B6B00111A75F00075A0787802E230E70700D5EE
:102B7B00F0F3022B8775A0787801EAF2D0F022C02F
:102B8B00F030111975F00075A0787802E230E70784
:102B9B0000D5F0F3022BA875A0787803E2D0F022D1
:102BAB00F22222AE82AF83902200EA2323232582D6
:102BBB00F58274003583F583E0F8A3E0F9EA245E2F
:102BCB00F5A089F08E828F831230DDF2A308E8B571
:102BDB00F003022C22DBF1AE82AF83902200EA23BA
:102BEB0023232582F58274003583F583E8BA000F21
:102BFB00C2ACF0200804D208D299D2AC022C1CD261
:102C0B000BF0902064EA14540F2582F582E0D2E792
:102C1B00F0E48E828F832274FF8E828F8322AE82AA
:102C2B00AF83902200EA2323232582F5827400359B
:102C3B0083F583E0F8A3E0F9EA245EF5A089F08E32
:102C4B00828F831230DDB4F308DB1C0BA3E8022C5C
:102C5B00DCB4F408DB330BA3E8022CDCB4F56EDB3D
:102C6B004A0BA3E8022CDCA31230DDB4F303022CD5
:102C7B00D814A3C082C08390250B2582F582E0D0A7
:102C8B0083D082122D32022CDCA31230DDB4F4037C
:102C9B00022CD814A3C082C08390250B2582F58209
:102CAB00E0D083D082122D83022CDCA31230DDB452
:102CBB00F503022CD814A3C082C08390250B258268
:102CCB00F582E0D083D082122D2E022CDC122D2E19
:102CDB00A3B5F006022D27022C4EDBFBAE82AF8391
:102CEB00902200EA2323232582F58274003583F595
:102CFB0083E8BA000FC2ACF0200804D208D299D2F4
:102D0B00AC022D21D20BF0902064EA14540F2582D3
:102D1B00F582E0D2E7F0E48E828F832274FF8E82FD
:102D2B008F8322F208E8227F017E20C39464400C3B
:102D3B001F7E31C394644004C394640E2464BE208C
:102D4B0002800EC0E0EE122D2EB5F003022D82D0C4
:102D5B00E07E31C3940A40030E80F81E240AC0E0C3
:102D6B00BE3003EF700AEE122D2EB5F003022D824A
:102D7B00D0E02430122D2E227F017E30C39464408C
:102D8B000C1F7E31C394644004C394640E2464C04E
:102D9B00E0EE122D2EB5F003022DD0D0E07E31C324
:102DAB00940A40030E80F81E240AC0E0BE3005EFE3
:102DBB0060027E30EE122D2EB5F003022DD0D0E046
:102DCB002430122D2E22200B03022E729000121291
:102DDB0030D1F5F0A31230D1F58385F082A3E582D3
:102DEB002411F582E5833400F583AE82AF83902006
:102DFB006475A0707A00C082C0838E828F8312307C
:102E0B00D154E0B4E007D083D082022E5AD083D0C5
:102E1B0082E030E73AC2E7F0EAC4032402F8C0824A
:102E2B00C0838E828F831230D1B40A168FF07465F3
:102E3B00F27FD7C2AFDFFE7475F27F24DFFED2AF15
:102E4B00AFF0D083D08274A5F20808087406F2A301
:102E5B00C082C0838E828F83A3AE82AF83D083D098
:102E6B00820ABA0191C20B228D828E83A3A31230E8
:102E7B00DD14540FC40375A0702402F8A31230DDC7
:102E8B00F9C2AF7465F274A5F27FDEE9DFFED9FCFF
:102E9B00F97475F27F6FDFFED9FC74B5F2D2AF22F5
:102EAB0090000A1230D1C2079000091230D1B40041
:102EBB000875366A753508801CB401087536877538
:102ECB0035E98011B40308753670753508800675C1
:102EDB00368875350885368C85358AC2AAD2A9D233
:102EEB000222E54E7003022F8F854E4F7A007B0036
:102EFB007800792A7D0075F026754520754400858C
:102F0B004582854483121375AE82AF837405258287
:102F1B00F58274003583F5837C04C204C20512303C
:102F2B00D1A36002D2041230D1A3B4FF028002D22B
:102F3B0005DCEB30041788828983EEF0A3EFF0A356
:102F4B00E54EC3954FF0A3A3A882A9830B300519B7
:102F5B008D8285F083EEF0A3EFF0A3E54EC3954F82
:102F6B00F0A3A3AD828583F00A854582854483A3B4
:102F7B00A3858245858344D54F8590257EEBF090C4
:102F8B00257DEAF022C2A878087A007B0190001216
:102F9B001230D1F5F0A31230D1F58385F082A31254
:102FAB0030D1F523A3AE82AF83E5822410F582E501
:102FBB00833400F5831230D1FD75A021BD0006745A
:102FCB0000D2E78055BD05067402D2E7804CBD06E2
:102FDB00067402D2E78043BD0C067401D2E7803A37
:102FEB00BDE0067404D2E78031BD0D067405D2E74F
:102FFB008028BD11067409D2E7801FBD0E06740729
:10300B00C2E78016BD0F067406D2E7800DBD100611
:10301B007408D2E780047403C2E7F2FCE82402F9D7
:10302B0075A022ECF3BDE0030230A375A070EA2477
:10303B0000F909097410F319197402A21EB392E076
:10304B00BD00028003BD0E0444188011A21BB39275
:10305B00E4A21C92E2A21D5004C2E4D2E3F3740773
:10306B00301F02740FF3EA2401F99030B9E52354B1
:10307B0007FC93F3EA2404F97488BC06028008BDAC
:10308B0005028003BD06027408F3EA2402F97401F9
:10309B00F3EA2405F97404F38F838E82E82408F88D
:1030AB00EA2408FADB028003022FAAD2A822446684
:1030BB008899BBCCCCBBC083C0E0E5832480F5836F
:1030CB00D0E0F0D08322C083E5832480F583E0D069
:1030DB008322300D04E4938011300A03E0800BC08F
:1030EB0083E5832480F583E0D08322C0D0C0E0C089
:1030FB0083C08275D010D55003755010E538B400DD
:10310B0004D2B480041538C2B4E537B40004D2B588
:10311B0080041537C2B5300211D201B294853E83BB
:10312B00853F82A385833E85823F200710C28CE5B5
:10313B008A2535F58AE58C3536F58CD28CD082D044
:10314B0083D0E0D0D032C0D0C0E0C083C082C01FDB
:10315B0075D018209811309903023225D01FD082D8
:10316B00D083D0E0D0D032C298E5874440F5873089
:10317B009F2AC29F902100E0547FB400117401F08C
:10318B00E58754BFF587759840D29C0231A7740030
:10319B00F0E58754BFF5877598C0D29CE58754BF7F
:1031AB00F587902100E0547FB400030231CEA3E0F9
:1031BB00F58275835CE599F00582E582902101F03B
:1031CB00023222902101E0F8A3E0F9A3E0FAA3E098
:1031DB00FBE599FF309A1030E70DC29A7B01E8FAB4
:1031EB000AEA6970027B00EB602175835C8A82EFCF
:1031FB00F00582E5826970047B00800FAA820B3098
:10320B009A098882EB14F0EAF87B00902101E8F030
:10321B00A3A3EAF0A3EBF002315EC29910140302F0
:10322B00322F215E902200E0F8A3E0B5180CE49059
:10323B002203F0A3F0C20802315EF8902100E054A3
:10324B007FB40031E8F8902204E0701275835E8839
:10325B0082E0902203F0902201E004F08011F890BC
:10326B002203E014B5180CE4902203F0A314F0D25F
:10327B009B8002C29B902201E075835EF582E0F594
:10328B00990582E582902201F0A3A3A3E004F0024A
:10329B00315EC0D0C0E0C0F0C083C08275D018755D
:1032AB003C01753D00753B00E53B9070052582F5B3
:1032BB0082E020E203023387C0E0902108E53B2542
:1032CB0082F582E0FCA385823A858339547FB40072
:1032DB000E907001E53B2582F582E0A2E5920C9001
:1032EB007003E53B2582F582E0F5F0EC20E7030265
:1032FB003385547FB40003023325853A82853983A5
:10330B00E0F582E53D245DF583E5F0F00582E5828D
:10331B00853A82853983F0023385853A82853983F4
:10332B00E0FCA3E0FDA3E0FEA3E0FFE5F0300C1012
:10333B0030E70DC20C7F01ECFE0EEE6D70027F00CC
:10334B00EF60258E82E53D245DF583E5F0F0058287
:10335B00E5826D70047F00800FAE820F300C098CFC
:10336B0082EF14F0EEFC7F00902109E53B2582F5FE
:10337B0082ECF0A3A3EEF0A3EFF0D0E020E0030289
:10338B0034C4902208E53D2323232582F582E0FFF8
:10339B00A3E0B51F22A3A37400F0A3F0907002E585
:1033AB003B2582F58274B1F0907005E53B2582F5E3
:1033BB00827404F00234C4F5F085823A858339A314
:1033CB00E0547FB400028008B4070280030234A0EB
:1033DB00C0E0A3E0FC600114FEA3E0FDD0E0B40765
:1033EB0005BC00538003BC001FE5F0F582E53D24CE
:1033FB005FF583E0FC0582E582853A82853983F0AF
:10340B00F5F0B51F070233A0EDB51E2B907002E54A
:10341B003B2582F5827415F0907000E53B2582F513
:10342B0082E0FEA3A37415F0907000E53B2582F5B6
:10343B0082EE4404F08029907002E53B2582F582F0
:10344B007415F0907000E53B2582F582E0FEA3A396
:10345B007415F0907000E53B2582F582EE54FBF07D
:10346B00E5F0F582E53D245FF583E0FE0582E5821C
:10347B00853A82853983F00DECB51D047C007D0007
:10348B00A3A3ECF0A3EDF0907003E53B2582F5824E
:10349B00EEF00234C4E5F0F582E53D245FF583E000
:1034AB00F5F00582E582853A82853983F0907003C9
:1034BB00E53B2582F582E5F0F0053DE53B2408F57B
:1034CB003BD53C0280030232B3D082D083D0F0D004
:1034DB00E0D0D0327480906003F07402906000F002
:1034EB007400906001F07407906003F074C19060F9
:1034FB0002F07400906001F07400906004F0906032
:10350B0005E0906006E022EFB54002800302387CB4
:10351B008D828E83A31230DDFCA31230DDFAA31251
:10352B0030DDFBBC07077F007901023836BC090E82
:10353B007F00A31230DDF970027901023836BC0826
:10354B0012A31230DDF9A31230DDFF4970027901AD
:10355B00023836BC1D077F00790102383BBC1F0EB9
:10356B007F00A31230DDF97002790102383BBC1EDB
:10357B0012A31230DDF9A31230DDFF49700279017D
:10358B0002383BBC5121EA541FFA240BF875A025D5
:10359B00E29401FAEB541FFB240BF875A025E2FB18
:1035AB007F007901023836BC521FEA541FFA240BF4
:1035BB00F875A025E2FAEB541FFB240BF875A02538
:1035CB00E2FB7F00790102383BBC5333EA541FFA0C
:1035DB00240BF875A025E29401FAEB541FFB240B86
:1035EB00F875A025E2FB7F00A31230DDF9541FF91B
:1035FB00240BF875A025E2F970027901023836BC6C
:10360B005431EA541FFA240BF875A025E2FAEB5457
:10361B001FFB240BF875A025E2FB7F00A31230DD06
:10362B00F9541FF9240BF875A025E2F97002790102
:10363B0002383BBC552CEA541FFA240BF875A02515
:10364B00E29401FAEB541FFB240BF875A025E2FB67
:10365B00A31230DDF9A31230DDFF497002790102AC
:10366B003836BC562AEA541FFA240BF875A025E20B
:10367B00FAEB541FFB240BF875A025E2FBA31230C9
:10368B00DDF9A31230DDFF497002790102383BBC32
:10369B00573CEA541FFA240BF875A025E29401FA63
:1036AB00EB541FFB240BF875A025E2FB7F00A31244
:1036BB0030DDF9541FF9240BF875A025E2F975F0EC
:1036CB001EA4F9E5F0FF4970027901023836BC58A7
:1036DB003AEA541FFA240BF875A025E2FAEB541FB3
:1036EB00FB240BF875A025E2FB7F00A31230DDF95C
:1036FB00541FF9240BF875A025E2F975F01EA4F9F7
:10370B00E5F0FF497002790102383BBC5913EB54C9
:10371B001FFB240BF875A025E2FB7F007901023813
:10372B0036BC5A13EB541FFB240BF875A025E2FB98
:10373B007F00790102383BBC5B25EB541FFB240B4C
:10374B00F875A025E2FB7F00A31230DDF9541FF9B9
:10375B00240BF875A025E2F970027901023836BC0A
:10376B005C25EB541FFB240BF875A025E2FB7F00B7
:10377B00A31230DDF9541FF9240BF875A025E2F9DB
:10378B007002790102383BBC5D1EEB541FFB240B0E
:10379B00F875A025E2FBA31230DDF9A31230DDFF93
:1037AB004970027901023836BC5E1EEB541FFB24B4
:1037BB000BF875A025E2FBA31230DDF9A31230DD67
:1037CB00FF497002790102383BBC5F2EEB541FFBA3
:1037DB00240BF875A025E2FB7F00A31230DDF95412
:1037EB001FF9240BF875A025E2F975F01EA4F9E575
:1037FB00F0FF4970027901023836BC6174EB541F3B
:10380B00FB240BF875A025E2FB7F00A31230DDF93A
:10381B00541FF9240BF875A025E2F975F01EA4F9D5
:10382B00E5F0FF497002790102383B904C008003B0
:10383B00905400EA75F008A42582F582E5F03583F3
:10384B00F583EBF0A3E0C39B5002F404BF000A899D
:10385B00F0B5F0004003848003F5F0E4C0E0A3E48E
:10386B00F0A3F0A3EFF0A3E9F0A3D0E0F0A3E5F011
:10387B00F022C290C2AFE4906000F0906005E0309F
:10388B00E5FC7447906003F0E4906000F0906005F5
:10389B00E030E6FC7407906003F0D2AF000000004C
:1038AB000000E4906000F0904C00753100C215E010
:1038BB00F532A3E0B5320AA3A3A3A3A3A3A30239B2
:1038CB00934064F532A3E0F551A3E0F552A3E0F584
:1038DB0055A3E0F556A3E0F553A3E0F554C3E53249
:1038EB009553F532E5542552F55274003551F55187
:1038FB00B55505E552B55600400E1532E5529556B5
:10390B00F552E5519555F551C3E5829406F582E5DF
:10391B00839400F583E532F0A3E551F0A3E552F073
:10392B00A3A3A3A3A38061F532A3E0F551A3E0F514
:10393B0052A3E0F555A3E0F556A3E0F553A3E0F54C
:10394B0054E5532532F532E5542552F552740035C2
:10395B0051F551B55505E552B55600400E0532E50A
:10396B00529556F552E5519555F551C3E58294069E
:10397B00F582E5839400F583E532F0A3E551F0A3DE
:10398B00E552F0A3A3A3A3A3C083C082906005E07C
:10399B0030E5FC906000E532F0D082D0831531E544
:1039AB003160030238BAB2153015030238BAD2901F
:1039BB0022008040C020A060E0109050D030B0704A
:1039CB00F0088848C828A868E8189858D838B878F4
:1039DB00F8048444C424A464E4149454D434B47418
:1039EB00F40C8C4CCC2CAC6CEC1C9C5CDC3CBC7C94
:1039FB00FC028242C222A262E2129252D232B27212
:103A0B00F20A8A4ACA2AAA6AEA1A9A5ADA3ABA7A93
:103A1B00FA068646C626A666E6169656D636B676B7
:103A2B00F60E8E4ECE2EAE6EEE1E9E5EDE3EBE7E33
:103A3B00FE018141C121A161E1119151D131B171DE
:103A4B00F1098949C929A969E9199959D939B97963
:103A5B00F9058545C525A565E5159555D535B57587
:103A6B00F50D8D4DCD2DAD6DED1D9D5DDD3DBD7D03
:103A7B00FD038343C323A363E3139353D333B37381
:103A8B00F30B8B4BCB2BAB6BEB1B9B5BDB3BBB7B03
:103A9B00FB078747C727A767E7179757D737B77727
:103AAB00F70F8F4FCF2FAF6FEF1F9F5FDF3FBF7FA3
:103ABB00FF15B115B11407140D14131419141F1499
:103ACB00B514B514B514BB14C114251431146714F3
:103ADB006D14731485145B143D144314491455145D
:103AEB004F148B14911497149D14AF14B514B51473
:103AFB00B51587158D14C714CD1599159F14611421
:103B0B003714D314D914DF14E514EB14F114F7158F
:103B1B00211527152D15331539153F1545154B1542
:103B2B0051157B1581159314A915A51D6D1E591ED5
:103B3B00DC14A315B1142B1479147F14FD15031584
:103B4B0009150F1515151B1557155D1563156915FA
:103B5B006F157514B514B514B514B514B514B51497
:103B6B00B514B514B514B514B514B514B514B51402
:103B7B00B515AB14B515B115B115B115B115B11509
:103B8B00B112444D58204D616368696E65205636FD
:103B9B002E35320D0020444D58204D616368696EFF
:103BAB00652076362E353220202020202000204123
:103BBB006C636F726E204D634272696465200020E6
:103BCB0053686F7720646174613A206261642000EE
:103BDB002053686F7720646174613A20206F6B20EB
:103BEB000020466C61672042616E6B2023203120E0
:103BFB002020466C61672042616E6B2023203220AF
:103C0B002020466C61672042616E6B20232033209D
:103C1B002020466C61672042616E6B20232034208C
:103C2B00205374617465205661726961626C652002
:103C3B002357616974696E6720666F72202020209C
:103C4B002020202020202020202020202020202069
:103C5B002020202020202020200065787465726EA3
:103C6B00616C2073796E632E2E2E20202020202055
:103C7B002020202020202020202020202020202039
:103C8B0020200045787465726E616C2073796E63C9
:103C9B002020202020202020202020202020202019
:103CAB002020202020202020202020007265636F00
:103CBB0076657265642E2020202020202020202075
:103CCB0020202020202020202020202020202020E9
:053CDB00202020200064
:00000001FF
